:10000000E3EF17F00000000000EF00F00000000038
:0A0010000000000000000000F3D71C
:10001C0092C1C9FFC7B002D00000FCD7C9CF01F014
:06002C0001C000F012000B
:040032008B821200AB
:10003600F250026EF29E0500FF6A0150FE6E0050FD
:08004600FD6E02BEF28E1200F5
:04004E008B9212007F
:10005200FDDF400E01018F11006E51C0E1FF52C061
:10006200E2FF00C0E6FF4FC000F050C001F0E2DF47
:1000720051C0E1FF52C0E2FF90C1E6FF4FC000F065
:1000820050C001F0D7DF51C0E1FF52C0E2FF91C181
:10009200E6FF4FC000F050C001F0CCDFC9DF120014
:1000A200D5DF51C0E1FF52C0E2FF7A0EE66E4FC0CB
:1000B20000F050C001F0BEDF51C0E1FF52C0E2FFCC
:1000C2008CC1E6FF4FC000F050C001F0B3DFB0DFDB
:0200D20012001A
:1000D40001018F6B8CC190F18DC191F1B8DFB5DF57
:1000E40051C0E1FF52C0E2FF3A0EE66E4FC000F08D
:1000F40050C001F09EDF51C0E1FF52C0E2FFE66A4A
:100104004FC000F050C001F094DF00C08EF18FDFCB
:060114008EC100F0120094
:10011A0099DFA00E01018C11006E51C0E1FF52C09F
:10012A00E2FF00C0E6FF4FC000F050C001F07EDFE2
:10013A0051C0E1FF52C0E2FF8DC1E6FF4FC000F09F
:0A014A0050C001F073DF70DF1200F7
:10015400020E01018F6F8CC190F18DC191F177DF97
:1001640074DF51C0E1FF52C0E2FF7A0EE66E4FC069
:1001740000F050C001F05DDF51C0E1FF52C0E2FF6A
:100184008EC1E6FF4FC000F050C001F052DF4FDFD8
:02019400120057
:100196005BDF51C0E1FF52C0E2FF8CC1E6FF4FC0FA
:1001A60000F050C001F044DF51C0E1FF52C0E2FF51
:1001B600E66A4FC000F050C001F03ADF00C08DF192
:0801C60035DF8DC100F01200CD
:1001CE003FDF800E01018C11006E51C0E1FF52C065
:1001DE00E2FF00C0E6FF4FC000F050C001F024DF88
:1001EE0051C0E1FF52C0E2FF8DC1E6FF4FC000F0EB
:0A01FE0050C001F019DF16DF1200F7
:10020800086A080E0C6E003408360450085ED8B030
:0E02180002D00826D89000360C2EF5D7120022
:10022600010182518025846F83518121856F010EE2
:10023600845F000E855B100E8F6F80C190F181C1C7
:1002460091F104DF120E01018F6F84C190F185C117
:1002560091F1FCDE1F0E01018C6F300E8D6FB4DF45
:100266001F0E01018C6F94DF200E0014016E0150E9
:0A027600000A02E00000F4D71200B5
:10028000086A096A100E0C6E0134083609360450EB
:10029000085E0550D8A0053C095ED8B007D00450D0
:1002A00008260550D8B0053C0926D89000360136FE
:0602B0000C2EEAD712003B
:1002B60080C18CF181C18DF182C18EF148DF83C18D
:0602C6008CF1ECDE1200D9
:1002CC000101876B010E825F000E835B835119085D
:1002DC0002E18251AD08FF0ED8B0000E006E005046
:1002EC008615016E0150000A07E0872BAD0E825D6A
:1002FC00886F190E8359896F8751000A05E0AD0E7E
:10030C008A6F190E8B6F04D082C18AF183C18BF175
:10031C0081518B1902E18A5180190DE180C18CF158
:10032C0081C18DF1D1DE00C08EF184C18CF185C10B
:10033C008DF10ADF30D0100E01018F6F80C190F16A
:10034C0081C191F180DE120E01018F6F8AC190F193
:10035C008BC191F178DE140E01018F6F84C190F185
:10036C0085C191F170DE1F0E01018C6F100E8D6F27
:10037C00CEDE1F0E01018C6F200E8D6F22DF1F0E43
:10038C0001018C6F02DF200E0014016E0150000A77
:10039C0002E00000F4D701018751000A1AE08051F5
:1003AC00825D006E81518359016E0050842701508B
:1003BC0085238851845F8951855B844B852B010E85
:1003CC00885D826F000E8959836F806B816B876BA0
:0403DC0093D71200A1
:1003E00036DE51C0E1FF52C0E2FF7A0EE66E4FC02A
:1003F00000F050C001F01FDE51C0E1FF52C0E2FF2B
:1004000081C1E6FF4FC000F050C001F014DE51C0C2
:10041000E1FF52C0E2FF80C1E6FF4FC000F050C0D4
:0804200001F009DE06DE120006
:10042800AE0E01018C6F190E8D6F8E6B8FDEAE0EC6
:1004380001018025006E190E8121016E00C080F136
:1004480001C081F1060E8F6F00C090F101C091F1DB
:10045800FCDD1F0E01018C6F800E8D6FB4DE1F0E48
:1004680001018C6F800E8D6F54DE00018651050AE4
:10047800FF0ED8A4000E016E8651070AFF0ED8A4FD
:10048800000E006E0150001206E01C0E01018C6F78
:100498000A0E8D6F3EDE1F0E01018C6F080E8D6FE8
:1004A80092DE00018651050AFF0ED8A4000E016EE7
:1004B8008651070AFF0ED8A4000E006E01500012E4
:1004C800D8B4ADD00101846B856B1C0E8C6F5FDED8
:1004D8000A0E00160050000AFF0ED8A4000E016E86
:1004E800030E0101855D02E1E80E845DFF0ED8B0C0
:1004F800000E006E005001160150000A03E0844B04
:10050800852BE3D71C0E8C6F42DE020E00160050BE
:10051800000A000ED8A4FF0E016E030E0101855DCE
:1005280002E1E80E845D000ED8B0FF0E006E0150A7
:100538000012D8B473D01F0E8C6F080E8D6FE9DDD2
:10054800040E010180258C6F000E81218D6FBEDDA8
:1005580000C083F10101866B1C0E8C6F18DE020E41
:1005680000160050000A000ED8A4FF0E016E006AA3
:10057800010183AB02D0FF0E006E0050011601503E
:10058800000A45E01F0E8C6F800E8D6F1CDE1F0E5B
:1005980001018C6F800E8D6FBCDD1C0E01018C6F0C
:1005A8000A0E8D6FB6DD1F0E01018C6F080E8D6F60
:1005B8000ADE0101846B856B1C0E8C6FE8DD0A0E68
:1005C80000160050000AFF0ED8A4000E016E030E9C
:1005D8000101855D02E1E80E845DFF0ED8B0000ED2
:1005E800006E0150001603E0844B852BE5D71F0EE3
:1005F8008C6F080E8D6F8DDD040E010180258C6FC8
:10060800000E81218D6F62DD00C083F101D006D01C
:10061800010186510F0A02E0862B9ED70CD00101FA
:100628001F0E8C6FB4DD080E0014016E0150000A15
:1006380002E00000F4D71D0E01018C6FA8DD060E44
:100648000014016E0150000A03E00101826B03D01F
:0C0658000101010E826F82C100F012004F
:10066400F4DC51C0E1FF52C0E2FF7A0EE66E4FC0E7
:1006740000F050C001F0DDDC01018251831117E06C
:1006840051C0E1FF52C0E2FF80C1E9FF81C1EAFF2E
:10069400EECFE6FF4FC000F050C001F0CADC01010C
:1006A400804B812B010E825F000E835BE5D7BFDC9C
:0206B400120032
:1006B600020E01018F6F80C190F181C191F1C6DCFC
:1006C600C3DC51C0E1FF52C0E2FF7A0EE66E4FC0B6
:1006D60000F050C001F0ACDC0101866B000E8519FC
:1006E60002E1000E841918E086518225E96E000E9B
:1006F6008321EA6E51C0E1FF52C0E2FFEECFE6FF72
:100706004FC000F050C001F093DC0101862B010EB2
:0C071600845F000E855BE2D789DC1200D6
:1007220095DC51C0E1FF52C0E2FF3A0EE66E4FC0C7
:1007320000F050C001F07EDC51C0E1FF52C0E2FF88
:10074200E66A4FC000F050C001F074DC00C06FF1E7
:080752006FDC6FC100F0120022
:10075A00AF0E0101806F190E816F6FC182F170C1F6
:10076A0083F1060E846F000E856FA0DF490E806F3D
:10077A00000E816F060E826F000E836F6EDF000E11
:10078A00806F080E816F27DE1C0E010177257D6FB1
:10079A00000E78217E6F000E806F450E816F1BDE82
:1007AA007DC180F17EC181F116DE7AC180F17BC103
:1007BA0081F111DE01017A4B7B2B806B816B0BDEA1
:1007CA00110E0101806F800E816F05DE0101806BC1
:1007DA00816B01DE740E0101806F000E816F040EC1
:1007EA00826F000E836F39DF71C180F172C181F1AE
:1007FA00040E826F000E836F30DF080E77257D6F3F
:10080A00000E78217E6F73C180F174C181F1E3DD3E
:10081A0075C180F176C181F1DEDD7DC180F17EC1D5
:10082A0081F1D9DD0101806B816BD5DDBD0E01013E
:10083A00806F190E816F140E826F000E836FEEDCCB
:10084A00160E01018C6FA2DC00C07FF1170E0101A8
:10085A008C6F9CDC00C082F1C70E0101806F190EFB
:10086A00816F7FC183F122DD010E01017D157C6F4D
:10087A00D90E77258C6F190E78218D6F8E6B65DCFA
:10088A00C90E0101806F190E816FD10E826F190E88
:10089A00836FD90E7725846F190E7821856F7C5165
:1008AA008427000E8523866B0CDDD90E7725806F91
:1008BA00190E7821816F7C518027000E8123080E42
:1008CA008027000E8123826B110E836FEFDC7EC1BD
:1008DA008CF151EC00F07DC18CF151EC00F0D10E9D
:1008EA000101806F190E816F0C0E7D25826F000E3B
:1008FA007E21836F7C518227000E83238FDC160EA4
:10090A0001018C6F43DC00C07FF1170E01018C6F6F
:10091A003DDC00C082F1D70E0101806F190E816F94
:10092A007FC183F1C3DC2A0E01017725806F000E97
:10093A007821816F74DD00C079F179C100F012006D
:10094A0027EC00F051C0E1FF52C0E2FF7A0EE66EDA
:10095A004FC000F050C001F01BEC00F001017251D1
:10096A00731120E051C0E1FF52C0E2FF6FC1F6FFF0
:10097A0070C1F7FF71C1F8FF0900F5CF00F000C0A0
:10098A00E6FF4FC000F050C001F01BEC00F0010E72
:10099A0001016F27000E70237123010E725F000E92
:0A09AA00735BDCD719EC00F01200BB
:1009B4006FC101F070C102F071C103F072C104F0A3
:1009C400000E0101741902E1000E731913E0010E07
:1009D400735F000E745B03C0E9FF04C0EAFF01C04B
:1009E400E1FF02C0E2FFEECFE6FF014A022A034A1A
:0609F400042AE6D7120000
:1009FA0001017251FF0A02E1FF0E711907E08F6BC4
:100A0A0071C190F172C191F129EC00F027EC00F06C
:100A1A0051C0E1FF52C0E2FF3A0EE66E4FC000F04D
:100A2A0050C001F01BEC00F0000E0101741902E144
:100A3A00000E731919E051C0E1FF52C0E2FFE66AE5
:100A4A004FC000F050C001F01BEC00F06FC1E1FF95
:100A5A0070C1E2FF00C0E6FF01016F4B702B010E6F
:0E0A6A00735F000E745BE0D719EC00F0120011
:100A78006FC104F070C105F071C106F072C107F0D2
:100A8800026A036A000E0101741902E1000E73196B
:100A980022E0010E735F000E745B04C0E9FF05C01D
:100AA800EAFFEECF00F0000E016E06C0D9FF07C0C6
:100AB800DAFFDE50005C026E000E0158036E000E75
:100AC800031802E1000E021801E005D0044A052AC5
:100AD800064A072AD7D702C000F003C001F0120067
:0C0AE800DE5003E0E66E74EF05F0120033
:100AF40070C1E1FF71C1E2FF200EE66E200EE66ECA
:100B0400300EE66EE66A020E01017025726F000E69
:100B14007121736F6F51000A1CE00A0E046E6FC1DD
:100B240000F004EC01F008C000F072C1E1FF73C1F1
:100B3400E2FF300E0024E66E0A0E046E6FC100F070
:100B440004EC01F000C06FF1010E725F000E735BE4
:040B5400E1D71200D3
:100B58000101716B726B27EC00F051C0E1FF52C0CC
:100B6800E2FF7A0EE66E4FC000F050C001F01BECB9
:100B780000F06FC1E9FF70C1EAFFEECF73F1010128
:100B88007351000A18E051C0E1FF52C0E2FF73C17F
:100B9800E6FF4FC000F050C001F01BEC00F001016F
:100BA800714B722B6F4B702B6FC1E9FF70C1EAFF5D
:100BB800EECF73F1E4D719EC00F071C100F072C107
:040BC80001F0120026
:100BCC0001016F513908000ED8B0FF0E016E300EC6
:100BDC006F5D000ED8B0FF0E006E00500114026E57
:060BEC0002C000F012003F
:100BF20071C1E1FF72C1E2FF200EE66E200EE66EC9
:100C0200200EE66E200EE66E300EE66EE66A040EEA
:100C120001017125736F000E7221746F000E70193D
:100C220002E1000E6F1929E00A0E046E000E056E35
:100C32006FC100F070C101F040EC01F008C000F09B
:100C420009C001F0300E002673C1E1FF74C1E2FF5A
:100C520000C0E6FF0A0E046E000E056E6FC100F0C2
:100C620070C101F040EC01F000C06FF101C070F101
:0C0C7200010E735F000E745BD1D71200FE
:100C7E000101726B736B27EC00F051C0E1FF52C0A3
:100C8E00E2FF7A0EE66E4FC000F050C001F01BEC92
:100C9E0000F06FC1F6FF70C1F7FF71C1F8FF0900D8
:100CAE00F5CF74F101017451000A1EE051C0E1FF4D
:100CBE0052C0E2FF74C1E6FF4FC000F050C001F019
:100CCE001BEC00F00101724B732B010E6F27000E0F
:100CDE00702371236FC1F6FF70C1F7FF71C1F8FF6A
:100CEE000900F5CF74F1DED719EC00F072C100F0F7
:060CFE0073C101F01200B9
:100D04000101406B416B000E3B1902E1500E3A1990
:100D140003E0406B416B59D2426B436BBA0E506F88
:100D2400000E516F42515027D8B0512BF8DC50C1FE
:100D3400E1FF51C1E2FF00C0E6FF000E01014319CB
:100D440002E10A0E421903E0424B432BE7D7BA0EE5
:100D5400E16E000EE26E4251E126D8B0E22AE66A64
:100D6400426B436B440E006E010E016E425100242F
:100D7400E16E000E0120E26E090E4225F66E340E7D
:100D8400F76E000EF722000EF86E000EF82209002E
:100D9400F5CF00F000C0E6FF000E431902E1040E97
:100DA400421903E0424B432BDDD7BA0E6F6F000E9E
:100DB400706F440E716F010E726F050E736F000E2B
:100DC400746F58DE000E011802E1000E001803E0F3
:100DD400406B416BFAD10001EA4BEB2BBF51730A14
:100DE400D8A4D8D0C90E01016F6F330E706F000EF6
:100DF400716F43DF00C040F101C041F1E90E6F6F34
:100E0400330E706F000E716F38DF005040270150B1
:100E140041230001C96BE86BE96BE8C001F0010EE6
:100E2400006E015004E000360090FF0FFBD7005025
:100E34008114016E006A015202E0010E006E00018D
:100E440000C0B0F0000EB16F000EB11902E1010E46
:100E5400B01917E1500EE16E010EE26EC90ED96EA3
:100E6400000EDA6E3FDE310EE66EE66AC90EE16E02
:100E7400000EE26E500ED96E010EDA6E33DEE66AB3
:100E840016D0500EE16E010EE26EC90ED96E000E40
:100E9400DA6E28DE300EE66EE66AC90EE16E000EEA
:100EA400E26E500ED96E010EDA6E1CDEE66A000E9A
:100EB400E91902E1070EE81903E0E84BE92BADD785
:100EC400C90E01016F6F000E706F44DE00504027A1
:100ED400015041230001C96BE86BE96BE8C001F0E4
:100EE400010E006E015004E000360090FF0FFBD7A6
:100EF40000508314016E006A015202E0010E006E7C
:100F040000C0B0F0000EB16F000EB11902E1010E85
:100F1400B01917E1500EE16E010EE26EC90ED96EE2
:100F2400000EDA6EDFDD310EE66EE66AC90EE16EA2
:100F3400000EE26E500ED96E010EDA6ED3DDE66A53
:100F440016D0500EE16E010EE26EC90ED96E000E7F
:100F5400DA6EC8DD300EE66EE66AC90EE16E000E8A
:100F6400E26E500ED96E010EDA6EBCDDE66A000E3A
:100F7400E91902E1070EE81903E0E84BE92BAED7C3
:100F8400C90E01016F6F000E706FE4DD0050402741
:100F9400015041230001BF51740AD8A4EED0C0C04F
:100FA4006FF112DE0050000A10E0300E0001C05D47
:100FB400006E00C001F0010E006E015004E0003626
:100FC4000090FF0FFBD70050831AC90E01016F6F09
:100FD400330E706F000E716F50DE00C040F101C01F
:100FE40041F1E90E6F6F330E706F000E716F45DEC5
:100FF40000504027015041230001C96BE86BE96BA5
:10100400E8C001F0010E006E015004E000360090CB
:10101400FF0FFBD700508114016E006A015202E0F9
:10102400010E006E000100C0B0F0000EB16F000EA2
:10103400B11902E1010EB01917E1500EE16E010E73
:10104400E26EC90ED96E000EDA6E4CDD310EE66E1C
:10105400E66AC90EE16E000EE26E500ED96E010E04
:10106400DA6E40DDE66A16D0500EE16E010EE26ED5
:10107400C90ED96E000EDA6E35DD300EE66EE66A04
:10108400C90EE16E000EE26E500ED96E010EDA6EDC
:1010940029DDE66A000EE91902E1070EE81903E00A
:1010A400E84BE92BADD7C90E01016F6F000E706FCD
:1010B40051DD00504027015041230001C96BE86B0A
:1010C400E96BE8C001F0010E006E015004E0003647
:1010D4000090FF0FFBD700508314016E006A015289
:1010E40002E0010E006E00C0B0F0000EB16F000E01
:1010F400B11902E1010EB01917E1500EE16E010EB3
:10110400E26EC90ED96E000EDA6EECDC310EE66EBC
:10111400E66AC90EE16E000EE26E500ED96E010E43
:10112400DA6EE0DCE66A16D0500EE16E010EE26E75
:10113400C90ED96E000EDA6ED5DC300EE66EE66AA4
:10114400C90EE16E000EE26E500ED96E010EDA6E1B
:10115400C9DCE66A000EE91902E1070EE81903E0AA
:10116400E84BE92BAED7C90E01016F6F000E706F0B
:10117400F1DC00504027015041230101000E4119C8
:1011840002E1000E401921E1C90E6F6F330E706F3A
:10119400000E716F72DD00C040F101C041F1E90E33
:1011A4006F6F330E706F000E716F67DD0050402754
:1011B40001504123700E6F6F310E706F000E716F0E
:1011C4005CDD005040270150412340C100F041C183
:0411D40001F0120014
:1011D800020E0C6E490E0D6E0D2EFED70C2EFCD78E
:0611E800000000001200EF
:1011EE0001013E6B3F6B36C1E9FF37C1EAFFEECF1F
:1011FE006FF1C90E706F000E716F75DC2E0E00014F
:10120E00CC6F010E01013625E96E000E3721EA6E14
:10121E00EECF6FF1400E706F010E716F64DC40C146
:10122E00CDF041C1CEF042C1CFF02E0E0001D06FF5
:10123E00020E01013625E96E000E3721EA6EEECF61
:10124E006FF1400E706F010E716F4DDC40C1D1F029
:10125E0041C1D2F042C1D3F02E0E0001D46F030E65
:10126E0001013625E96E000E3721EA6EEECF6FF1E1
:10127E00400E706F010E716F36DC40C1D5F041C16A
:10128E00D6F042C1D7F03A0E0001D86F38C16FF1D7
:10129E0039C170F1400E0101716F010E726FA2DC47
:1012AE0040C1D9F041C1DAF042C1DBF043C1DCF0FC
:1012BE0044C1DDF05B0E0001DE6F3AC16FF13BC140
:1012CE0070F1400E0101716F010E726F8BDC40C127
:1012DE00DFF041C1E0F042C1E1F043C1E2F044C1B0
:1012EE00E3F05D0E0001E46FE56B1C0E01013C2581
:1012FE003E6F000E3D213F6FC90E806F000E816F55
:10130E001C0E826F000E836F32EC03F0000E3D193F
:10131E0002E1000E3C190CE091EC03F000C08CF1E0
:10132E0051EC00F0010E01013C5F000E3D5BEED76B
:0A133E003EC100F03FC101F01200B3
:101348000101396B3C0E00019C6F000E9D6F9E6F72
:101358009F6F91EC03F000C037F10050020AD8A447
:1013680029D10101386B91EC03F0010138510E0AC3
:1013780002E0382BF8D7A80E6F6F000E706FFF0EC3
:10138800716FFF0E726F040E736F000E746FFDECB9
:1013980004F0386B91EC03F001013851070A02E0C0
:1013A800382BF8D7386B91EC03F000C037F1490EB1
:1013B800D96E000EDA6E01013851D926D8B0DA2A72
:1013C8000050DE1801E021D13851050A02E0382B1F
:1013D800EAD7386B91EC03F001013851CD0A02E0ED
:1013E800382BF8D73A6B01013A51000AD8A4E2D059
:1013F80091EC03F000C037F10050350A0EE191EC92
:1014080003F000C037F10050010A05E191EC03F048
:1014180000C039F101D0F9D0CCD001013751010A0F
:1014280019E191EC03F000C037F10050040A10E113
:10143800A40E01016F6F000E706FFF0E716FFF0E2B
:10144800726F040E736F000E746FFDEC04F001D020
:10145800DCD0AFD001013751030A24E191EC03F04D
:1014680000C037F1040E005C10E3A00E01016F6F9D
:10147800000E706FFF0E716FFF0E726F040E736FA8
:10148800000E746FFDEC04F001D0BFD00101040E12
:10149800375F3751000A05E091EC03F00101370787
:1014A800F8D787D03751060A24E191EC03F000C041
:1014B80037F1040E005C10E38C0E01016F6F000E13
:1014C800706FFF0E716FFF0E726F040E736F000E58
:1014D800746FFDEC04F001D098D00101040E375F61
:1014E8003751000A05E091EC03F001013707F8D7FE
:1014F80060D03751360A19E191EC03F000C037F19A
:101508000050040A10E13B0E01016F6F010E706F6D
:10151800FF0E716FFF0E726F040E736F000E746F03
:10152800FDEC04F001D071D044D001013751FF0A1D
:1015380003E1010E3A6F3DD03751330A2DE191ECAA
:1015480003F000C037F10050040A24E19C0E0101A9
:101558006F6F000E706FFF0E716FFF0E726F040ECB
:10156800736F000E746FFDEC04F000019F510008CA
:1015780008E19E51000805E19D51070802E19C51D0
:10158800080807E2080E9C5F070E9D5B000E9E5B35
:101598009F5B01D03AD00DD091EC03F000C037F139
:1015A80001013751000A05E091EC03F0010137070A
:1015B800F7D719D701013951020A0FE17E0E6F6F73
:1015C800000E706F3B0E716F010E726F040E736F19
:1015D800000E746FDAEC04F015D07E0E6F6F000EFB
:1015E800706F3B0E716F010E726F040E736F000EF9
:1015F800746F3CEC05F0000E011802E1000E0018B3
:1016080001E0396B39C136F102D00101366B36C1C0
:0416180000F01200CC
:10161C00980E01016F6F000E706F36C171F137C1FA
:10162C0072F1040E736F000E746FDAEC04F0940E0A
:10163C006F6F000E706F38C171F139C172F1040E09
:10164C00736F000E746FDAEC04F0900E6F6F000E77
:10165C00706F3AC171F13BC172F1040E736F000EE1
:08166C00746FDAEC04F01200C7
:1016740036C101F037C102F0000E01013A1902E14E
:10168400000E39190DE0010E395F000E3A5B01C0FE
:10169400E1FF02C0E2FF38C1E6FF014A022AECD7AB
:0216A400120032
:1016A600F90E01013A6F000E3B6F020E8F6FD90ED5
:1016B600906F190E916F29EC00F0F70E01016F6F14
:1016C600330E706F000E716F0C0E726F000E736F1B
:1016D600A5EC04F03651030AFF0ED8A4000E016EE5
:1016E6003751000A000ED8A4FF0E006E01500016F6
:1016F6000BE0A80E806F000E816F040E826F000E45
:10170600836F32EC03F00AD0396B8C6B51EC00F02E
:1017160001013951030A02E0392BF7D7396B8C6B7B
:1017260051EC00F0010139510B0A02E0392BF7D7D1
:10173600490E806F000E816F060E826F000E836F5A
:1017460032EC03F0396B8C6B51EC00F0010139512E
:10175600C90A02E0392BF7D7030E6F6F340E706F8C
:10176600000E716F060E726F000E736FA5EC04F01B
:1017760036C18CF151EC00F001013651030AFF0E1F
:10178600D8A4000E016E3751000AFF0ED8A4000E31
:10179600006E015000161CE0360E8C6F51EC00F006
:1017A600040E01018C6F51EC00F07E0E0101806F7A
:1017B600000E816F040E826F000E836F32EC03F011
:1017C6003A4B3B2B3A4B3B2B040E3A27000E3B235E
:1017D6000F0E6F6F340E706F000E716F050E726F05
:1017E600000E736FA5EC04F03651030AFF0ED8A461
:1017F600000E016E3751000AFF0ED8A4000E006ECF
:101806000150001625E0320E8C6F51EC00F0040EEC
:1018160001018C6F51EC00F00101396BA80EE96EE5
:10182600000EEA6E3951E926D8B0EA2AEECF8CF1DD
:1018360051EC00F001013951030A02E0392BEED7D1
:101846003A4B3B2B3A4B3B2B040E3A27000E3B23DD
:10185600FF0E8C6F51EC00F06D0E01016F6F000EE4
:10186600706F6D0E716F000E726F440E736F000E07
:10187600746F430E756F000E766F3AC177F13BC1F8
:1018860078F1ADEC03F000C038F138C100F0120079
:1018960027EC00F0400E01012C11006E51C0E1FF53
:1018A60052C0E2FF00C0E6FF4FC000F050C001F09A
:1018B6001BEC00F051C0E1FF52C0E2FF2DC1E6FF74
:1018C6004FC000F050C001F01BEC00F019EC00F026
:0218D6001200FE
:1018D80001018C6BCBEC00F000C033F1010E01016B
:1018E8008C6FCBEC00F000C034F101018F6B2CC180
:1018F80090F12DC191F129EC00F027EC00F051C0D6
:10190800E1FF52C0E2FF3A0EE66E4FC000F050C051
:1019180001F01BEC00F00101326B3051000A19E0B4
:1019280051C0E1FF52C0E2FFE66A4FC000F050C06C
:1019380001F01BEC00F0010132512E25D96E000E8A
:101948002F21DA6E0050DE1801E003D0322B300769
:10195800E4D719EC00F08F6B33C190F134C191F1E9
:0E19680029EC00F030C131F131C100F0120065
:10197600B50E0101806F190E816FBB0E826F190EB5
:10198600836FAF0E846F190E856F866B66EC01F060
:10199600B50E806F190E816F490E826F000E836F30
:0E19A600060E846F000E856F5BEC03F01200DE
:1019B400C90E0101806F190E816FCD0E826F190E51
:1019C400836FCD0E846F190E856F866B66EC01F004
:1019D400C90E806F190E816F740E826F000E836FB3
:0E19E400040E846F000E856F5BEC03F01200A2
:1019F20001012C6BECEC08F0ECEC08F02C51C70A5E
:081A020002E02C2BF7D71200C3
:101A0A001F0E01018C6F010E8D6F8DEC00F01F0E01
:0E1A1A0001018C6F020E8D6FE7EC00F01200E0
:101A280091EC03F091EC03F091EC03F000C02DF180
:101A380091EC03F000C02CF191EC03F000C02FF101
:101A480091EC03F000C02EF191EC03F000C031F1ED
:101A580091EC03F000C030F191EC03F091EC03F04D
:101A680091EC03F091EC03F001012E512F1114E0D9
:101A780091EC03F00050000A01E0FAD791EC03F072
:101A880091EC03F091EC03F091EC03F0010E0101ED
:101A98002E5F000E2F5BE8D7000E311902E1000E11
:101AA80030194CE091EC03F091EC03F091EC03F069
:101AB80000C035F191EC03F000C034F191EC03F073
:101AC80091EC03F091EC03F091EC03F091EC03F04E
:101AD80091EC03F091EC03F000C033F191EC03F0CA
:101AE80000C032F1000E0101351902E1010E34196E
:101AF80011E191EC03F000C0B6F091EC03F000C0E6
:101B0800B7F091EC03F000C0B8F091EC03F000C01E
:101B1800B9F014D0000E0101331902E1000E321998
:101B280008E091EC03F0010E0101325F000E335B17
:0E1B3800F1D7010E305F000E315BAED7120008
:101B460001012D51190802E12C51AD0804E2AE0E37
:101B56002C5F190E2D5B8F6B2CC190F12DC191F16D
:061B660029EC00F0120062
:101B6C000B6A0A6A096A00500402F4CF09F0F3CF39
:101B7C0008F001500502F4CF0BF0F3CF0AF000503F
:101B8C000502F3500926F4500A22E86A0B22015090
:101B9C000402F3500926F4500A22E86A0B2208C00A
:101BAC0000F009C001F00AC002F00BC003F01200F3
:101BBC007350020A1AE1740E0101366F000E376F72
:101BCC00386B040E396F000E3A6F4EDD010E366F16
:101BDC00376B63DD43C0B2F044C0B3F045C0B4F022
:101BEC0046C0B5F0030E736E9ED07350030A24E109
:101BFC00050E0001B225016E000EB321026E000E1F
:101C0C00B421036E000EB521046E4650045C08E14D
:101C1C004550035C05E14450025C02E14350015C19
:101C2C0002E2020E736EA4EC09F00050020A03E10A
:101C3C00040E736E04D077D07350040A10E1030EB7
:101C4C00366F65C037F129DD43C0B2F044C0B3F044
:101C5C0045C0B4F046C0B5F0050E736E64D0735039
:101C6C00050A35E1A4EC09F000C02CF10050060A7D
:101C7C0003E1040E736E2AD02C51050A27E143C0F0
:101C8C00B2F044C0B3F045C0B4F046C0B5F0060E97
:101C9C00736E740E6F6F000E706FA80E716F000E66
:101CAC00726F040E736F000E746FDAEC04F0A40EF6
:101CBC00366F000E376FA00E386F000E396F8C0E1A
:101CCC003A6F000E3B6FA4DC656A2DD02CD073509C
:101CDC00060A29E1010E0001B225016E000EB321A6
:101CEC00026E000EB421036E000EB521046E04507A
:101CFC00465C08E10350455C05E10250445C02E19E
:101D0C000150435C0FE30001010E9C5F000E9D5BD4
:101D1C009E5B9F5B43C0B2F044C0B3F045C0B4F0CF
:081D2C0046C0B5F000D0120022
:101D34001F0E01018C6F010E8D6F8DEC00F01F0ED4
:0E1D440001018C6F020E8D6F8DEC00F012000D
:101D52005BDE140E01012C6F09C12DF19BDD48DE03
:101D6200160E2C6F0BC12DF195DD42DE170E2C6F76
:0A1D72000AC12DF18FDD3CDE1200E6
:101D7C000DC18CF10EC18DF16AEC00F000C012F1B6
:101D8C0091EC03F000C011F191EC03F000C010F1E4
:101D9C0091EC03F000C00FF10101176B1C6B010EED
:101DAC001D6F1A6B1B6B0C0E0D258C6F000E0E210C
:101DBC008D6F6AEC00F0040E016E00C015F1000E80
:101DCC000101166F015004E01533159FFF0FFBD76F
:101DDC00000E166F153715911637153715911637E6
:101DEC00270E6F6F010E706FC90E716F190E726F27
:101DFC00040E736F000E746FFDEC04F00D0E0D25C8
:101E0C008C6F000E0E218D6F6AEC00F0000E016ECF
:101E1C003F0E00140101136F01C014F1000E1417D2
:101E2C000E0E7C5C186F000E7D58196F0B51185FED
:101E3C000C51195B1551185F1651195B020E0D25CB
:101E4C008C6F000E0E218D6F6AEC00F000C08EF1CD
:101E5C000DC18CF10EC18DF1AAEC00F0030E010145
:101E6C000D258C6F000E0E218D6F6AEC00F000C0FA
:101E7C008CF151EC00F011C180F112C181F1F0EC48
:101E8C0001F0040E01010D258C6F000E0E218D6FDB
:101E9C006AEC00F000C07BF091EC03F000C07AF02B
:101EAC0091EC03F000C079F091EC03F000C078F0F5
:101EBC0091EC03F000C085F091EC03F000C084F0CD
:101ECC0091EC03F000C083F091EC03F000C082F0C1
:101EDC00000E0101141902E1020E131937E1010E73
:101EEC0078240001826F000E7920836F000E7A2017
:101EFC00846F000E7B20856F120E0101136F000E94
:101F0C00146F0C0E8C6FCBEC00F000C078F00D0E43
:101F1C0001018C6FCBEC00F000C079F001018C6BEF
:101F2C00CBEC00F000C07AF0010E01018C6FCBEC11
:101F3C0000F000C07BF00101172B140E156F000E82
:101F4C00166F1A6B1B6B00018B6B6DD0000E0101B1
:101F5C00141902E1180E13192FE178C01EF179C083
:101F6C001FF17AC020F17BC021F182C078F083C0D0
:101F7C0079F084C07AF085C07BF018511E250001E1
:101F8C00826F010119511F210001836F000E0101A5
:101F9C0020210001846F000E010121210001856FB9
:101FAC00100E0101136F000E146F172B140E156F0A
:101FBC00000E166F1C2B37D0000E141902E1110EF7
:101FCC00131931E178C01EF179C01FF17AC020F1EC
:101FDC007BC021F182C078F083C079F084C07AF0A4
:101FEC0085C07BF0010E1E250001826F000E0101E1
:101FFC001F210001836F000E010120210001846F5D
:10200C00000E010121210001856F100E0101136FDB
:10201C00000E146F172B140E156F000E166F1A6B23
:10202C001B6B00018B2B01011751000AD8B4A7D1EF
:10203C000101040E0D25806F000E0E21816F7BC0F7
:10204C0082F17AC083F15BEC01F079C08CF151EC38
:10205C0000F078C08CF151EC00F085C08CF151ECA3
:10206C0000F084C08CF151EC00F083C08CF151EC89
:10207C0000F082C08CF151EC00F00C0E01010D252A
:10208C008C6F000E0E218D6F6AEC00F00F0E001499
:10209C0001018E6F15C100F016C101F000360090E1
:1020AC00013600360090013600508E130C0E0D25B3
:1020BC008C6F000E0E218D6FAAEC00F00D0E01013D
:1020CC000D258C6F000E0E218D6F6AEC00F0C00E8A
:1020DC00001401018E6F13518E130D0E0D258C6F94
:1020EC00000E0E218D6FAAEC00F001010B511A2588
:1020FC00186F0C511B21196F1551182716511923E4
:10210C001D51000A02E031DC4FDCBF0E806F190E4E
:10211C00816F19C182F118C183F15BEC01F0C70E1C
:10212C000101806F190E816F826B836B5BEC01F088
:10213C00BD0E0101806F190E816F0BC182F10CC1B4
:10214C0083F113EC01F0160E01018C6FCBEC00F057
:10215C0000C02BF1170E01018C6FCBEC00F000C00E
:10216C0082F1C70E0101806F190E816F2BC183F1B3
:10217C005BEC01F0BD0E01011825236F190E19211E
:10218C00246F100E0D25806F000E0E21816F826B57
:10219C00836B5BEC01F0010E01011815226F23C15A
:1021AC008CF124C18DF18E6BAAEC00F0C90E0101EB
:1021BC00806F190E816FD10E826F190E836F2251B1
:1021CC002325846F000E2421856F866B66EC01F04D
:1021DC00080E2325806F000E2421816F2251802749
:1021EC00000E8123826B060E836F5BEC01F00A0EEE
:1021FC0001012325806F000E2421816F225180273D
:10220C00000E81231A511525036E1B511621046EE5
:10221C0004C000F0016A00C082F11A511525836FC9
:10222C005BEC01F00DC180F10EC181F101011A517D
:10223C001525826F1B511621836F0C0E8227000E01
:10224C00832322518227000E832313EC01F0160EF8
:10225C0001018C6FCBEC00F000C02BF1170E0101CB
:10226C008C6FCBEC00F000C082F1100E01010D253B
:10227C00806F000E0E21816F2BC183F15BEC01F09E
:10228C000E0E01011825806F000E1921816F14ECC0
:10229C0002F01C51000A58E0100E136F000E146F60
:1022AC001C6B1D6B020E8F6F15510D25906F165107
:1022BC000E21916F29EC00F00E0E010109252C6FF7
:1022CC00000E0A212D6F0B512C270C512D2315516B
:1022DC002C2716512D2331DC00018B2B270E026E7F
:1022EC00010E036E0E0E7C5C006E000E7D58016EAE
:1022FC0001010B51005E0C51015A1551005E165133
:10230C00015A89C0E1FF8AC0E2FF02C0E6FF03C0A8
:10231C00E6FF11C1E6FF12C1E6FF0FC1E6FF10C1D7
:10232C00E6FF00C0E6FF01C0E6FF8B0EE66E000E76
:10233C00E66E87C000F088C001F01BEC00F000C016
:10234C001AF101C01BF174D600018B51000A17E081
:10235C0001011A5178261B517922000E7A227B2218
:10236C00110E136F000E146F00018B6B01011D6BAE
:10237C00140E156F000E166F1A6B1B6B59D61200CC
:10238C000CC18CF10DC18DF16AEC00F000C011F1A3
:10239C0091EC03F000C010F191EC03F000C00FF1D0
:1023AC0091EC03F000C00EF1000E01010F1902E1D7
:1023BC00000E0E1901E19CD091EC03F000C013F15A
:1023CC0091EC03F000C012F11A0E01016F6F010EB7
:1023DC00706FC90E716F190E726F040E736F000E51
:1023EC00746FFDEC04F0020E8F6F080E0C25906FCD
:1023FC00000E0D21916F29EC00F00E0E0101092544
:10240C002C6F000E0A212D6F0B512C27000E2D2343
:10241C00080E2C27000E2D23A3EC0DF0000E01014D
:10242C00111902E1350E101903E114EC0DF060D016
:10243C00000E01010F1902E1440E0E1903E1DEEC4E
:10244C000DF056D01A0E026E010E036E080E01012D
:10245C00125D006E000E1359016E55C0E1FF56C09F
:10246C00E2FF02C0E6FF03C0E6FF10C1E6FF11C1A8
:10247C00E6FF0EC1E6FF0FC1E6FF00C0E6FF01C09C
:10248C00E6FF53C000F054C001F01BEC00F000C09C
:10249C0012F101C013F1000E026E0150025C02E158
:1024AC000050000825E2140E01016F6F010E706FD1
:1024BC00B50E716F190E726F060E736F000E746F7E
:1024CC00FDEC04F0140E6F6F010E706F1A0E716F2D
:1024DC00010E726F0EC173F10FC174F110C175F161
:1024EC0011C176F112C177F113C178F1ADEC03F0A3
:0224FC001200CC
:1024FE00C40E01018C6F190E8D6F6AEC00F000C0D6
:10250E0009F101010951010A5BE1D50E2C6F190E7B
:10251E002D6F740E2E6F000E2F6F040E306F6CEC3D
:10252E000CF00050000A4BE1C40E01018C6F190E25
:10253E008D6F020E8E6FAAEC00F0BBEC0CF0CB0E82
:10254E00806F190E816FCF0E826F190E836FD50EAD
:10255E00846F190E856F866B66EC01F0CB0E806F63
:10256E00190E816F740E826F000E836F040E846FCE
:10257E00000E856F5BEC03F0C50E806F190E816F38
:10258E00CB0E826F190E836FCF0E846F190E856F6F
:10259E00866B66EC01F0C50E806F190E816F490EC9
:1025AE00826F000E836F060E846F000E856F5BECDC
:1025BE0003F03C0E806F000E816F14EC02F09AD087
:1025CE0001010951020AD8A495D0AF0E2C6F190E35
:1025DE002D6F490E2E6F000E2F6F060E306F6CECA6
:1025EE000CF00050000AFF0ED8A4000E0101096F76
:1025FE00CB0E2C6F190E2D6F47C02EF148C02FF148
:10260E00040E306F6CEC0CF00050000AFF0ED8A4D4
:10261E00000E016E015001010915006E6AE042C004
:10262E0000F0000E016E0F0E046E000E056EB6EC7D
:10263E000DF0150E00246F6F000E0120706F090E45
:10264E006F27000E7023C50E716F190E726F060E76
:10265E00736F000E746FFDEC04F042C000F0000EBC
:10266E00016E0F0E046E000E056EB6EC0DF0150E1B
:10267E0000246F6F000E0120706F050E6F27000E85
:10268E00702347C071F148C072F1040E736F000ED3
:10269E00746FDAEC04F042C000F0000E016E0F0E03
:1026AE00046E000E056EB6EC0DF0150E0024E16EF4
:1026BE00000E0120E26E010EE66E42C000F0000E2A
:1026CE00016E0F0E046E000E056EB6EC0DF0150EBB
:1026DE000026000E0122010E0024E16E000E0120E4
:1026EE00E26E43C0E6FF44C0E6FF45C0E6FF46C0CB
:0626FE00E6FF00D012000F
:1027040005EC0DF0140E01012C6F09C12DF14BECF9
:102714000CF0120E01018C6F010E8D6FE7EC00F0CE
:10272400F9EC0CF0120E8C6F010E8D6F8DEC00F035
:10273400160E01018C6FCBEC00F00CC1E1FF0DC152
:10274400E2FF00C0E6FF170E01018C6FCBEC00F036
:0E2754000AC1E1FF0BC1E2FF00C0E6FF120068
:102762001F0E01018C6F010E8D6FE7EC00F01F0E42
:0E27720001018C6F020E8D6FE7EC00F012007B
:102780000001FE51000A07E001012C6B0D0E2D6FB8
:102790004BEC0CF006D001012C6B010E2D6F4BECB5
:1027A0000CF00001FE51000A08E0020E01012C6F3E
:1027B000310E2D6F4BEC0CF007D0020E01012C6F87
:1027C000300E2D6F4BEC0CF00A0E01018F6FEE0EE8
:1027D000906F050E916F29EC00F00001FE51000A88
:1027E00008E0040E01012C6F150E2D6F4BEC0CF060
:1027F00007D0040E01012C6F120E2D6F4BEC0CF064
:10280000060E01012C6F120E2D6F4BEC0CF0000127
:10281000FE51000A07E1070E01012C6F0C0E2D6F0F
:102820004BEC0CF00001FE51000A07E1090E01011A
:102830002C6F3F0E2D6F4BEC0CF093DF040E01015B
:102840002C6F49C02DF14BEC0CF0050E01012C6FE3
:102850004AC02DF14BEC0CF0020E01012C6F4BC065
:102860002DF14BEC0CF0030E01012C6F4CC02DF13F
:102870004BEC0CF001012C6B4DC02DF14BEC0CF02E
:10288000010E01012C6F4EC02DF14BEC0CF0150E1A
:1028900001012C6F2D6B4BEC0CF0120E01018C6FB3
:1028A000CBEC00F000C086F00101096BFF0E0A6F4F
:1028B000000E0B6F000E0C6F010E0D6F23DF000179
:1028C000FE51000A0DE00101096BFE0E0001FF152B
:1028D00001010A6F0A8100C10BF1A9EC0EF00BD0C7
:1028E0000101096BFE0E0001FF1501010A6F00C115
:1028F0000BF1A9EC0EF0100E096F010E0A6F0B6BB5
:10290000A9EC0EF01F0E8C6F040E8D6FE7EC00F03B
:10291000F9EC0CF0150E366F000E376F386B2D0E7C
:10292000396F000E3A6F3AEC0BF09AEC0EF0120091
:102930001F0E01018C6F010E8D6FE7EC00F01F0E72
:0E29400001018C6F020E8D6F8DEC00F0120005
:10294E000001FE6B9AEC0EF001018F6B57C090F1F7
:10295E0058C091F129EC00F027EC00F051C0E1FFD6
:10296E0052C0E2FF3A0EE66E4FC000F050C001F0CA
:10297E001BEC00F051C0E1FF52C0E2FFE66A4FC00F
:10298E0000F050C001F01BEC00F000C057F051C039
:10299E00E1FF52C0E2FFE66A4FC000F050C001F006
:1029AE001BEC00F000C058F051C0E1FF52C0E2FF36
:1029BE00E66A4FC000F050C001F01BEC00F000C002
:1029CE007CF051C0E1FF52C0E2FFE66A4FC000F05A
:1029DE0050C001F01BEC00F000C07DF051C0E1FFD3
:1029EE0052C0E2FFE66A4FC000F050C001F01BEC8F
:1029FE0000F000C003F151C0E1FF52C0E2FFE66AF1
:102A0E004FC000F050C001F01BEC00F000C004F10C
:102A1E0019EC00F0040E7C5C036E000E7D58046E03
:102A2E0003C07CF004C07DF05850190802E15750E5
:102A3E00AD08FF0ED8B0000E026E010E5714016ED7
:102A4E000150000A000ED8A4FF0E006E00500212B4
:102A5E00800E01010415016E0150000A000ED8A46B
:102A6E00FF0E006E00500210016E0450050802E1C8
:102A7E000350EE08FF0ED8B0000E006E005001108D
:102A8E00026E800E0315016E0150000AFF0ED8A4CF
:102A9E00000E006E0250001204E0010E0001FE6FE7
:102AAE00B5D101018C6BCBEC00F000C001F1010E31
:102ABE0001018C6FCBEC00F000C002F101C180F17E
:102ACE0002C181F17C5001010125826F7D500221EE
:102ADE00836FAF0E846F190E856F010E866F66ECD5
:102AEE0001F0BB0E8C6F190E8D6F6AEC00F000C0FA
:102AFE0004F191EC03F000C003F101010451080A46
:102B0E0002E1060E031911E1BD0E2C6F190E2D6F89
:102B1E00660E2E6F000E2F6F070E306F6CEC0CF0E2
:102B2E000050000A01E1E4DC49D101010451080A18
:102B3E0002E1000E0319D8A43ED1CD0E2C6F190E52
:102B4E002D6F740E2E6F000E2F6F040E306F6CEC07
:102B5E000CF00050000A000ED8A4FF0E0101006F09
:102B6E00CD0E2C6F190E2D6F6D0E2E6F000E2F6F5A
:102B7E00040E306F6CEC0CF00050000A000ED8A45E
:102B8E00FF0E016E015001010015006E04E0020EF1
:102B9E000001FE6F0FD1BD0E01018C6F190E8D6FEE
:102BAE006AEC00F0F00E0014016E0150400A04E0D1
:102BBE00030E0001FE6FFED0BD0E01018C6F190ECB
:102BCE008D6F6AEC00F000C005F1000E0101066F7A
:102BDE000F0E0517000E0617053705910637053738
:102BEE0005910637C30E8C6F190E8D6F6AEC00F0CF
:102BFE00BF0E00160050000AFF0ED8A4000E0101F1
:102C0E00006FC40E8C6F190E8D6F6AEC00F00050C1
:102C1E00000AFF0ED8A4000E016E0101005101162C
:102C2E000150000AD8B4C6D0BD0E0525076F190E87
:102C3E000621086FC60E8C6F190E8D6F6AEC00F0B0
:102C4E0000C0FFF00050010AD8A491D007C18CF14A
:102C5E0008C18DF16AEC00F00050080AFF0ED8A4EE
:102C6E00000E0101006F010E07258C6F000E08216A
:102C7E008D6F6AEC00F00050000AFF0ED8A4000E13
:102C8E00016E015001010015006E70E007C18CF15C
:102C9E0008C18DF18E6BAAEC00F0BBEC0CF0DAECF7
:102CAE000CF0C70E806F190E816F826B836B5BEC1D
:102CBE0001F0BD0E0101806F190E816F05C182F109
:102CCE0006C183F113EC01F0160E01018C6FCBECF3
:102CDE0000F000C000F1170E01018C6FCBEC00F07C
:102CEE0000C082F1C70E0101806F190E816F00C105
:102CFE0083F15BEC01F0020E01010725806F000EDF
:102D0E000821816F826B836B5BEC01F007C180F150
:102D1E0008C181F1010105517C5C826F06517D581D
:102D2E00836F0E0E825F000E835B13EC01F0160EA6
:102D3E0001018C6FCBEC00F000C000F1170E010109
:102D4E008C6FCBEC00F000C082F1020E0101072562
:102D5E00806F000E0821816F00C183F15BEC01F0E2
:102D6E007CC080F17DC081F114EC02F023D0000113
:102D7E00FF51110A0DE101C109F102C10AF105C1AC
:102D8E000BF107C10CF108C10DF1C6EC11F012D018
:102D9E000001FF51060A0EE101C109F102C10AF15B
:102DAE0005C10BF106C10CF107C10DF108C10EF101
:102DBE00BEEC0EF003D0040E0001FE6F1E0E0101DC
:102DCE008C6F400E8D6FE7EC00F0010E575C016EBC
:102DDE00000E5858026E0250190802E10150AD085B
:102DEE000AE20C0E01018F6FAD0E906F190E916FEE
:102DFE0029EC00F00BD00C0E01018F6F010E575C09
:102E0E00906F000E5858916F29EC00F0FEC000F044
:022E1E001200A0
:102E2000A69CF6C0A9FFA69EA680A8CF01F001C06F
:042E300000F012009C
:102E3400C69A1C0E4F6E000E506E920E516E010E0D
:102E4400526EFF0E0001AC6FFF0EAD6FFF0EAE6F42
:102E5400FF0EAF6F949A94969488C66A400EC76E1C
:042E6400C68A120008
:102E680094908B80949219EC00F0F9EC0CF08B9014
:102E7800F9EC0CF08B80F9EC0CF027EC00F051C069
:102E8800E1FF52C0E2FFFF0EE66E4FC000F050C0F7
:102E980001F01BEC00F019EC00F0F9EC0CF0490E15
:102EA8006F6F000E706FF6C071F1F7C072F1060E09
:102EB800736F000E746FDAEC04F0740E6F6F000E0F
:102EC800706FF8C071F1F9C072F1040E736F000EE3
:102ED800746FDAEC04F0666A010E676E080E686EAD
:102EE800696A060E6A6E040E6B6E6C6A6D0E366F3A
:102EF800000E376FFF0E386F060E396F000E3A6FEF
:102F08003AEC0BF0436A446A456A466A426A736A55
:102F1800656A576A586A9AEC0EF0080E01018F6FBD
:102F2800906B916B29EC00F00A0E01018F6FAD0ECA
:102F3800906F190E916F29EC00F00C0E01018F6F44
:102F4800AD0E906F190E916F29EC00F001018F6B97
:102F5800906B916B29EC00F0040E01018F6FAE0E9F
:102F6800906F190E916F29EC00F005EC0DF0FAC086
:062F7800FEF002DC120075
:102F7E00F6C087F0F7C088F0F8C089F0F9C08AF083
:102F8E00FAC053F0FBC054F0FCC055F0FDC056F033
:022F9E0012001F
:102FA0000001F66BC5DC190E01018C6FCBEC00F053
:102FB0000050000803E2CBDC00C0F6F09AEC0EF003
:062FC000F6C000F0120053
:102FC6000B0EC16E806AFF0E926E816AFF0E936EC3
:102FD600836A956A0001EA6BEB6B100EF66F000EC2
:102FE600F76F1BDF00C0ECF0110EF66F000EF76FE7
:102FF60014DF00C0EDF0120EF66F000EF76F0DDF56
:1030060000C0EEF0130EF66F000EF76F06DF00C07D
:10301600EFF0140EF66F000EF76FFFDE00C0F0F053
:10302600150EF66F000EF76FF8DE00C0F1F0F66BC6
:10303600F76BF3DE00C0F2F0010EF66F000EF76FCD
:10304600ECDE00C0F3F0020EF66F000EF76FE5DE61
:1030560000C0F4F0030EF66F000EF76FDEDE00C060
:10306600F5F0040EF66F000EF76FD7DE00C061F0C4
:10307600050EF66F000EF76FD0DE00C062F0060E8A
:10308600F66F000EF76FC9DE00C063F0070EF66F2D
:10309600000EF76FC2DE00C064F0080EF66F000E79
:1030A600F76FBBDE00C05DF0090EF66F000EF76F1E
:1030B600B4DE00C05EF00A0EF66F000EF76FADDEEE
:1030C60000C05FF00B0EF66F000EF76FA6DE00C0B5
:1030D60060F00C0EF66F000EF76F9FDE00C059F021
:1030E6000D0EF66F000EF76F98DE00C05AF00E0E4A
:1030F600F66F000EF76F91DE00C05BF00F0EF66FF5
:10310600000EF76F8ADE00C05CF091DEEC0EF66F03
:10311600000EF76FF20EF86F000EF96F010EFA6FE0
:10312600A0DE040E0001F66F0D0EF76F360EF86F77
:10313600010EF96FEE0EFA6F110EFB6F360EFC6F75
:10314600010EFD6F19DF590E0101366F000E376F44
:10315600610E386F000E396F5D0E3A6F000E3B6FD1
:0A3166000EEC0BF01ADFFED7FFD7C6
:103170003C6D65746120687474702D657175697635
:103180003D22726566726573682220636F6E746596
:103190006E743D22333B75726C3D687474703A2FC7
:1031A0002F79656C6C6F77646F6737372E6E6F2D74
:1031B00069702E62697A223E3C48544D4C3E3C4830
:1031C0004541443E3C2F484541443E3C424F4459D2
:1031D0003E3C68313E4D4355436F6E74726F6C20B8
:1031E00076312E303C2F68313E3C2F424F44593EC1
:1031F0003C2F48544D4C3E000000000000000000F1
:1032000000000000000000000000000000000000BE
:1032100000000000000000000000000000000000AE
:10322000000000000000000000000000000000009E
:10323000000000000000000000000000000000008E
:10324000000000000000000000000000000000007E
:10325000000000000000000000000000000000006E
:10326000000000000000000000000000000000005E
:10327000000000000000000000000000000000004E
:10328000000000000000000000000000000000003E
:10329000000000000000000000000000000000002E
:1032A000000000000000000000000000000000001E
:1032B000000000000000000000000000000000000E
:1032C00000000000000000000000000000000000FE
:1032D00000000000000000000000000000000000EE
:1032E00000000000000000000000000000000000DE
:1032F00000000000000000000000000000000000CE
:1033000000000000000000000000000000000000BD
:1033100000000000000000000000000000000000AD
:10332000000000000000000000000000000000009D
:10333000000000000000000000000000000000008D
:10334000000000000000000000000000000000007D
:10335000000000000000000000000000000000006D
:10336000000000000000000000000000000000005D
:10337000000000000000000000000000000000004D
:10338000000000000000000000000000000000003D
:10339000000000000000000000000000000000002D
:1033A000000000000000000000000000000000001D
:1033B000000000000000000000000000000000000D
:0933C00000000000000000000004
:1033C900485454502F312E3120323030204F4B0A7F
:1033D900436F6E74656E742D747970653A200000C0
:0E33E900746578742F68746D6C0A0A00000019
:0C33F70001010600122334450000800094
:06340300638253633501F2
:06340900474554202F008E
:05340F00370301030674
:020000040030CA
:0D000100220F0EFF0181FF0FC00FE00F4026
:00000001FF
